 battdrvr

 Timestamp is 4fb05c79 (Mon May 14 13:14:33 2012)

 Preferred load address is 10000000

 Start         Length     Name                   Class
 0001:00000000 00000004H .CRT$XCA                CODE
 0001:00000004 00000004H .CRT$XCZ                CODE
 0001:00000008 00000004H .CRT$XIA                CODE
 0001:0000000c 00000004H .CRT$XIZ                CODE
 0001:00000010 00000004H .CRT$XPA                CODE
 0001:00000014 00000004H .CRT$XPZ                CODE
 0001:00000018 00000004H .CRT$XTA                CODE
 0001:0000001c 00000004H .CRT$XTZ                CODE
 0001:00000020 00001068H .rdata                  CODE
 0001:00001088 00000025H .rdata$debug            CODE
 0001:000010b0 000031d8H .text                   CODE
 0001:00004288 00000118H .xdata                  CODE
 0001:000043a0 00000014H .idata$2                CODE
 0001:000043b4 00000014H .idata$3                CODE
 0001:000043c8 000000a8H .idata$4                CODE
 0001:00004470 0000000cH .idata$6                CODE
 0001:00004480 000000dcH .edata                  CODE
 0002:00000000 000000a8H .idata$5                DATA
 0002:000000a8 0000044cH .data                   DATA
 0002:00000500 000000f8H .bss                    DATA
 0003:00000000 000001f0H .pdata                  DATA

  Address         Publics by Value              Rva+Base       Lib:Object

 0000:00000000       ___safe_se_handler_table   00000000     <absolute>
 0000:00000000       ___safe_se_handler_count   00000000     <absolute>
 0001:00000000       __xc_a                     10001000     corelib0:crt0init.obj
 0001:00000004       __xc_z                     10001004     corelib0:crt0init.obj
 0001:00000008       __xi_a                     10001008     corelib0:crt0init.obj
 0001:0000000c       __xi_z                     1000100c     corelib0:crt0init.obj
 0001:00000010       __xp_a                     10001010     corelib0:crt0init.obj
 0001:00000014       __xp_z                     10001014     corelib0:crt0init.obj
 0001:00000018       __xt_a                     10001018     corelib0:crt0init.obj
 0001:0000001c       __xt_z                     1000101c     corelib0:crt0init.obj
 0001:0000003c       ??_C@_1DE@FPIJCBIJ@?$AA?9?$AAB?$AAa?$AAt?$AAt?$AAe?$AAr?$AAy?$AAP?$AAD?$AAD?$AAD?$AAe?$AAi?$AAn?$AAi?$AAt?$AAi?$AAa?$AAl?$AAi?$AAz?$AAe?$AA?$AN?$AA?6?$AA?$AA@ 1000103c     battdrvr.obj
 0001:00000070       ??_C@_1DE@PAFCCPOG@?$AA?$CL?$AAB?$AAa?$AAt?$AAt?$AAe?$AAr?$AAy?$AAP?$AAD?$AAD?$AAD?$AAe?$AAi?$AAn?$AAi?$AAt?$AAi?$AAa?$AAl?$AAi?$AAz?$AAe?$AA?$AN?$AA?6?$AA?$AA@ 10001070     battdrvr.obj
 0001:000000a4       ??_C@_1CI@KLFHNCOH@?$AA?9?$AAB?$AAa?$AAt?$AAt?$AAe?$AAr?$AAy?$AAP?$AAD?$AAD?$AAR?$AAe?$AAs?$AAu?$AAm?$AAe?$AA?$AN?$AA?6?$AA?$AA@ 100010a4     battdrvr.obj
 0001:000000cc       ??_C@_1CI@POCOLDPH@?$AA?$CL?$AAB?$AAa?$AAt?$AAt?$AAe?$AAr?$AAy?$AAP?$AAD?$AAD?$AAR?$AAe?$AAs?$AAu?$AAm?$AAe?$AA?$AN?$AA?6?$AA?$AA@ 100010cc     battdrvr.obj
 0001:000000f4       ??_C@_1DE@IMOPIBJ@?$AA?9?$AAB?$AAa?$AAt?$AAt?$AAe?$AAr?$AAy?$AAP?$AAD?$AAD?$AAP?$AAo?$AAw?$AAe?$AAr?$AAH?$AAa?$AAn?$AAd?$AAl?$AAe?$AAr?$AA?$AN?$AA?6?$AA?$AA@ 100010f4     battdrvr.obj
 0001:00000128       ??_C@_1DE@KHBFPGHG@?$AA?$CL?$AAB?$AAa?$AAt?$AAt?$AAe?$AAr?$AAy?$AAP?$AAD?$AAD?$AAP?$AAo?$AAw?$AAe?$AAr?$AAH?$AAa?$AAn?$AAd?$AAl?$AAe?$AAr?$AA?$AN?$AA?6?$AA?$AA@ 10001128     battdrvr.obj
 0001:0000015c       ??_C@_1CO@DDBIBLBI@?$AA?9?$AAB?$AAa?$AAt?$AAt?$AAe?$AAr?$AAy?$AAP?$AAD?$AAD?$AAG?$AAe?$AAt?$AAS?$AAt?$AAa?$AAt?$AAu?$AAs?$AA?$AN?$AA?6?$AA?$AA@ 1000115c     battdrvr.obj
 0001:0000018c       ??_C@_1CO@OINMEEDD@?$AA?$CL?$AAB?$AAa?$AAt?$AAt?$AAe?$AAr?$AAy?$AAP?$AAD?$AAD?$AAG?$AAe?$AAt?$AAS?$AAt?$AAa?$AAt?$AAu?$AAs?$AA?$AN?$AA?6?$AA?$AA@ 1000118c     battdrvr.obj
 0001:000001bc       ??_C@_1CO@OMPCNBHK@?$AA?9?$AAB?$AAa?$AAt?$AAt?$AAe?$AAr?$AAy?$AAP?$AAD?$AAD?$AAG?$AAe?$AAt?$AAL?$AAe?$AAv?$AAe?$AAl?$AAs?$AA?$AN?$AA?6?$AA?$AA@ 100011bc     battdrvr.obj
 0001:000001ec       ??_C@_1CO@DHDGIOFB@?$AA?$CL?$AAB?$AAa?$AAt?$AAt?$AAe?$AAr?$AAy?$AAP?$AAD?$AAD?$AAG?$AAe?$AAt?$AAL?$AAe?$AAv?$AAe?$AAl?$AAs?$AA?$AN?$AA?6?$AA?$AA@ 100011ec     battdrvr.obj
 0001:00000220       ??_C@_1FA@CNGJDKAB@?$AA?9?$AAB?$AAa?$AAt?$AAt?$AAe?$AAr?$AAy?$AAP?$AAD?$AAD?$AAS?$AAu?$AAp?$AAp?$AAo?$AAr?$AAt?$AAs?$AAC?$AAh?$AAa?$AAn?$AAg?$AAe?$AAN?$AAo?$AAt?$AAi?$AAf?$AAi?$AAc@ 10001220     battdrvr.obj
 0001:00000270       ??_C@_1FA@GFLIGKHP@?$AA?$CL?$AAB?$AAa?$AAt?$AAt?$AAe?$AAr?$AAy?$AAP?$AAD?$AAD?$AAS?$AAu?$AAp?$AAp?$AAo?$AAr?$AAt?$AAs?$AAC?$AAh?$AAa?$AAn?$AAg?$AAe?$AAN?$AAo?$AAt?$AAi?$AAf?$AAi?$AAc@ 10001270     battdrvr.obj
 0001:000002c0       ??_C@_1BM@OBNKDNPL@?$AA?$CF?$AAs?$AA?3?$AA?5?$AAe?$AAx?$AAi?$AAt?$AAi?$AAn?$AAg?$AA?$AN?$AA?6?$AA?$AA@ 100012c0     battdrvr_lib:battdrvr.obj
 0001:000002e0       ??_C@_1GE@MMCMIDCB@?$AA?$CF?$AAs?$AA?3?$AA?5?$AAW?$AAa?$AAi?$AAt?$AAF?$AAo?$AAr?$AAS?$AAi?$AAn?$AAg?$AAl?$AAe?$AAO?$AAb?$AAj?$AAe?$AAc?$AAt?$AA?$CI?$AA?$CJ?$AA?5?$AAr?$AAe?$AAt?$AAu?$AAr?$AAn@ 100012e0     battdrvr_lib:battdrvr.obj
 0001:00000344       ??_C@_1DC@MHFFDPEB@?$AA?$CF?$AAs?$AA?3?$AA?5?$AAs?$AAy?$AAs?$AAt?$AAe?$AAm?$AA?5?$AAh?$AAa?$AAs?$AA?5?$AAr?$AAe?$AAs?$AAu?$AAm?$AAe?$AAd?$AA?$AN?$AA?6?$AA?$AA@ 10001344     battdrvr_lib:battdrvr.obj
 0001:00000378       ??_C@_1HC@IJCKHMEA@?$AA?$CF?$AAs?$AA?3?$AA?5?$AAt?$AAh?$AAr?$AAe?$AAa?$AAd?$AA?5?$AAp?$AAr?$AAi?$AAo?$AAr?$AAi?$AAt?$AAy?$AA?5?$AAi?$AAs?$AA?5?$AA?$CF?$AAd?$AA?0?$AA?5?$AAt?$AAi?$AAm?$AAe?$AAo@ 10001378     battdrvr_lib:battdrvr.obj
 0001:000003f0       ??_C@_1FK@FNONLNGN@?$AA?$CF?$AAs?$AA?3?$AA?5?$AAD?$AAE?$AAB?$AAU?$AAG?$AAC?$AAH?$AAK?$AA?5?$AAf?$AAa?$AAi?$AAl?$AAe?$AAd?$AA?5?$AAi?$AAn?$AA?5?$AAf?$AAi?$AAl?$AAe?$AA?5?$AA?$CF?$AAs?$AA?5?$AAa@ 100013f0     battdrvr_lib:battdrvr.obj
 0001:00000450       ??_C@_1HK@GPKEAHHI@?$AAC?$AA?3?$AA?2?$AAy?$AAm?$AAz?$AAk?$AAi?$AA?2?$AAp?$AAu?$AAb?$AAl?$AAi?$AAc?$AA?2?$AAC?$AAO?$AAM?$AAM?$AAO?$AAN?$AA?2?$AAo?$AAa?$AAk?$AA?2?$AAd?$AAr?$AAi?$AAv?$AAe@ 10001450     battdrvr_lib:battdrvr.obj
 0001:000004cc       ??_C@_1DG@KKOCKJAD@?$AAB?$AAa?$AAt?$AAt?$AAe?$AAr?$AAy?$AA?3?$AA?5?$AAB?$AAa?$AAt?$AAt?$AAe?$AAr?$AAy?$AAT?$AAh?$AAr?$AAe?$AAa?$AAd?$AAP?$AAr?$AAo?$AAc?$AA?$AA@ 100014cc     battdrvr_lib:battdrvr.obj
 0001:00000504       ??_C@_1CG@EPNLEKEF@?$AA?$CF?$AAs?$AA?3?$AA?5?$AAr?$AAe?$AAt?$AAu?$AAr?$AAn?$AAi?$AAn?$AAg?$AA?5?$AA?$CF?$AAd?$AA?$AN?$AA?6?$AA?$AA@ 10001504     battdrvr_lib:battdrvr.obj
 0001:0000052c       ??_C@_1DO@FBABFCGB@?$AA?$CF?$AAs?$AA?3?$AA?5?$AAC?$AAr?$AAe?$AAa?$AAt?$AAe?$AAT?$AAh?$AAr?$AAe?$AAa?$AAd?$AA?$CI?$AA?$CJ?$AA?5?$AAf?$AAa?$AAi?$AAl?$AAe?$AAd?$AA?5?$AA?$CF?$AAd?$AA?$AN?$AA?6?$AA?$AA@ 1000152c     battdrvr_lib:battdrvr.obj
 0001:00000570       ??_C@_1IK@KCLDPPJD@?$AA?$CF?$AAs?$AA?3?$AA?5?$AAB?$AAa?$AAt?$AAt?$AAe?$AAr?$AAy?$AAP?$AAD?$AAD?$AAI?$AAn?$AAi?$AAt?$AAi?$AAa?$AAl?$AAi?$AAz?$AAe?$AA?$CI?$AA?$CJ?$AA?5?$AAf?$AAa?$AAi?$AAl?$AAe@ 10001570     battdrvr_lib:battdrvr.obj
 0001:00000600       ??_C@_1IA@ENLKDIEP@?$AA?$CF?$AAs?$AA?3?$AA?5?$AAB?$AAa?$AAt?$AAt?$AAe?$AAr?$AAy?$AAP?$AAD?$AAD?$AAI?$AAn?$AAi?$AAt?$AAi?$AAa?$AAl?$AAi?$AAz?$AAe?$AA?$CI?$AA?$CJ?$AA?5?$AAf?$AAa?$AAi?$AAl?$AAe@ 10001600     battdrvr_lib:battdrvr.obj
 0001:00000680       ??_C@_1BM@KBMAGFOO@?$AAP?$AAd?$AAd?$AAB?$AAu?$AAf?$AAf?$AAe?$AAr?$AAS?$AAi?$AAz?$AAe?$AA?$AA@ 10001680     battdrvr_lib:battdrvr.obj
 0001:0000069c       ??_C@_1BK@GMCBNGHD@?$AAP?$AAo?$AAl?$AAl?$AAI?$AAn?$AAt?$AAe?$AAr?$AAv?$AAa?$AAl?$AA?$AA@ 1000169c     battdrvr_lib:battdrvr.obj
 0001:000006b8       ??_C@_1CA@NFABIDNC@?$AAP?$AAo?$AAl?$AAl?$AAP?$AAr?$AAi?$AAo?$AAr?$AAi?$AAt?$AAy?$AA2?$AA5?$AA6?$AA?$AA@ 100016b8     battdrvr_lib:battdrvr.obj
 0001:000006d8       ??_C@_1EI@MONKPJMD@?$AA?$CF?$AAs?$AA?3?$AA?5?$AAB?$AAa?$AAt?$AAt?$AAe?$AAr?$AAy?$AAP?$AAD?$AAD?$AAI?$AAn?$AAi?$AAt?$AAi?$AAa?$AAl?$AAi?$AAz?$AAe?$AA?$CI?$AA?$CJ?$AA?5?$AAf?$AAa?$AAi?$AAl?$AAe@ 100016d8     battdrvr_lib:battdrvr.obj
 0001:00000720       ??_C@_1DG@BGHDBENB@?$AA?$CF?$AAs?$AA?3?$AA?5?$AAC?$AAr?$AAe?$AAa?$AAt?$AAe?$AAE?$AAv?$AAe?$AAn?$AAt?$AA?$CI?$AA?$CJ?$AA?5?$AAf?$AAa?$AAi?$AAl?$AAe?$AAd?$AA?$AN?$AA?6?$AA?$AA@ 10001720     battdrvr_lib:battdrvr.obj
 0001:00000758       ??_C@_1FA@HLFIBIAK@?$AA?$CF?$AAs?$AA?3?$AA?5?$AAf?$AAa?$AAt?$AAa?$AAl?$AA?5?$AAe?$AAr?$AAr?$AAo?$AAr?$AA?3?$AA?5?$AAc?$AAa?$AAn?$AA?8?$AAt?$AA?5?$AAo?$AAp?$AAe?$AAn?$AA?5?$AAA?$AAP?$AAI?$AA?5@ 10001758     battdrvr_lib:battdrvr.obj
 0001:000007a8       ??_C@_1DA@IBFGCKKH@?$AAS?$AAY?$AAS?$AAT?$AAE?$AAM?$AA?1?$AAB?$AAa?$AAt?$AAt?$AAe?$AAr?$AAy?$AAA?$AAP?$AAI?$AAs?$AAR?$AAe?$AAa?$AAd?$AAy?$AA?$AA@ 100017a8     battdrvr_lib:battdrvr.obj
 0001:000007d8       ??_C@_1EA@FGBOCLMM@?$AA?$CF?$AAs?$AA?3?$AA?5?$AAi?$AAn?$AAv?$AAo?$AAk?$AAe?$AAd?$AA?5?$AAw?$AA?1?$AA?5?$AAc?$AAo?$AAn?$AAt?$AAe?$AAx?$AAt?$AA?5?$AA0?$AAx?$AA?$CF?$AA0?$AA8?$AAx?$AA?$AN?$AA?6?$AA?$AA@ 100017d8     battdrvr_lib:battdrvr.obj
 0001:00000818       ??_C@_1BO@MBKJIGNO@?$AAB?$AAa?$AAt?$AAt?$AAD?$AAr?$AAv?$AAr?$AA?3?$AA?5?$AAI?$AAn?$AAi?$AAt?$AA?$AA@ 10001818     battdrvr_lib:battdrvr.obj
 0001:00000838       ??_C@_1DI@BDOBKKI@?$AAB?$AAa?$AAt?$AAt?$AAe?$AAr?$AAy?$AA?3?$AA?5?$AAD?$AAe?$AAi?$AAn?$AAi?$AAt?$AA?3?$AA?5?$AAa?$AAl?$AAl?$AA?5?$AAd?$AAo?$AAn?$AAe?$AA?$AN?$AA?6?$AA?$AA@ 10001838     battdrvr_lib:battdrvr.obj
 0001:00000870       ??_C@_1FK@PGLDMCNF@?$AAB?$AAa?$AAt?$AAt?$AAe?$AAr?$AAy?$AA?3?$AA?5?$AAD?$AAe?$AAi?$AAn?$AAi?$AAt?$AA?3?$AA?5?$AAi?$AAn?$AAv?$AAo?$AAk?$AAe?$AAd?$AA?5?$AAw?$AA?1?$AA?5?$AAc?$AAo?$AAn?$AAt@ 10001870     battdrvr_lib:battdrvr.obj
 0001:000008cc       ??_C@_1DK@KFJEDHHH@?$AA?$CF?$AAs?$AA?3?$AA?5?$AAr?$AAe?$AAt?$AAu?$AAr?$AAn?$AAi?$AAn?$AAg?$AA?5?$AA?$CF?$AAd?$AA?0?$AA?5?$AAe?$AAr?$AAr?$AAo?$AAr?$AA?5?$AA?$CF?$AAd?$AA?$AN?$AA?6?$AA?$AA@ 100018cc     battdrvr_lib:battdrvr.obj
 0001:00000908       ??_C@_1EA@EEDKECB@?$AA?$CF?$AAs?$AA?3?$AA?5?$AAU?$AAn?$AAs?$AAu?$AAp?$AAp?$AAo?$AAr?$AAt?$AAe?$AAd?$AA?5?$AAI?$AAO?$AAC?$AAT?$AAL?$AA?5?$AAc?$AAo?$AAd?$AAe?$AA?5?$AA?$CF?$AAu?$AA?$AN?$AA?6?$AA?$AA@ 10001908     battdrvr_lib:battdrvr.obj
 0001:00000948       ??_C@_1EI@OIHICLDC@?$AA?$CF?$AAs?$AA?3?$AA?5?$AAP?$AAD?$AAD?$AA?5?$AAI?$AAO?$AAC?$AAo?$AAn?$AAt?$AAr?$AAo?$AAl?$AA?$CI?$AA?$CF?$AAu?$AA?$CJ?$AA?5?$AAr?$AAe?$AAt?$AAu?$AAr?$AAn?$AAe?$AAd?$AA?5?$AA?$CF@ 10001948     battdrvr_lib:battdrvr.obj
 0001:00000990       ??_C@_1GI@EFENJIE@?$AA?$CF?$AAs?$AA?3?$AA?5?$AAe?$AAx?$AAc?$AAe?$AAp?$AAt?$AAi?$AAo?$AAn?$AA?5?$AAi?$AAn?$AA?5?$AAI?$AAO?$AAC?$AAT?$AAL?$AA_?$AAB?$AAA?$AAT?$AAT?$AAE?$AAR?$AAY?$AA_?$AAN@ 10001990     battdrvr_lib:battdrvr.obj
 0001:000009f8       ??_C@_1HI@FMLCHJCL@?$AA?$CF?$AAs?$AA?3?$AA?5?$AAe?$AAx?$AAc?$AAe?$AAp?$AAt?$AAi?$AAo?$AAn?$AA?5?$AAi?$AAn?$AA?5?$AAI?$AAO?$AAC?$AAT?$AAL?$AA_?$AAB?$AAA?$AAT?$AAT?$AAE?$AAR?$AAY?$AA_?$AAS@ 100019f8     battdrvr_lib:battdrvr.obj
 0001:00000a70       ??_C@_1FG@JCAPGPO@?$AA?$CF?$AAs?$AA?3?$AA?5?$AAe?$AAx?$AAc?$AAe?$AAp?$AAt?$AAi?$AAo?$AAn?$AA?5?$AAi?$AAn?$AA?5?$AAI?$AAO?$AAC?$AAT?$AAL?$AA_?$AAB?$AAA?$AAT?$AAT?$AAE?$AAR?$AAY?$AA_?$AAG@ 10001a70     battdrvr_lib:battdrvr.obj
 0001:00000ac8       ??_C@_1GC@LFOHNMPD@?$AA?$CF?$AAs?$AA?3?$AA?5?$AAe?$AAx?$AAc?$AAe?$AAp?$AAt?$AAi?$AAo?$AAn?$AA?5?$AAi?$AAn?$AA?5?$AAI?$AAO?$AAC?$AAT?$AAL?$AA_?$AAB?$AAA?$AAT?$AAT?$AAE?$AAR?$AAY?$AA_?$AAG@ 10001ac8     battdrvr_lib:battdrvr.obj
 0001:00000b30       ??_C@_1IO@MPHPACCJ@?$AA?$CF?$AAs?$AA?3?$AA?5?$AAe?$AAx?$AAc?$AAe?$AAp?$AAt?$AAi?$AAo?$AAn?$AA?5?$AAw?$AAr?$AAi?$AAt?$AAi?$AAn?$AAg?$AA?5?$AAs?$AAt?$AAa?$AAt?$AAu?$AAs?$AA?5?$AAi?$AAn?$AA?5@ 10001b30     battdrvr_lib:battdrvr.obj
 0001:00000bc0       ??_C@_1IO@MHLNDPLD@?$AA?$CF?$AAs?$AA?3?$AA?5?$AAe?$AAx?$AAc?$AAe?$AAp?$AAt?$AAi?$AAo?$AAn?$AA?5?$AAr?$AAe?$AAa?$AAd?$AAi?$AAn?$AAg?$AA?5?$AAs?$AAt?$AAa?$AAt?$AAu?$AAs?$AA?5?$AAi?$AAn?$AA?5@ 10001bc0     battdrvr_lib:battdrvr.obj
 0001:00000c50       ??_C@_1JA@IEBNKALF@?$AA?$CF?$AAs?$AA?3?$AA?5?$AAe?$AAx?$AAc?$AAe?$AAp?$AAt?$AAi?$AAo?$AAn?$AA?5?$AAw?$AAr?$AAi?$AAt?$AAi?$AAn?$AAg?$AA?5?$AAs?$AAt?$AAa?$AAt?$AAu?$AAs?$AA?5?$AAi?$AAn?$AA?5@ 10001c50     battdrvr_lib:battdrvr.obj
 0001:00000ce0       ??_C@_1JA@FHNLIGPG@?$AA?$CF?$AAs?$AA?3?$AA?5?$AAe?$AAx?$AAc?$AAe?$AAp?$AAt?$AAi?$AAo?$AAn?$AA?5?$AAr?$AAe?$AAa?$AAd?$AAi?$AAn?$AAg?$AA?5?$AAs?$AAt?$AAa?$AAt?$AAu?$AAs?$AA?5?$AAi?$AAn?$AA?5@ 10001ce0     battdrvr_lib:battdrvr.obj
 0001:00000d70       ??_C@_1IO@DBOPPHKG@?$AA?$CF?$AAs?$AA?3?$AA?5?$AAe?$AAx?$AAc?$AAe?$AAp?$AAt?$AAi?$AAo?$AAn?$AA?5?$AAr?$AAe?$AAa?$AAd?$AAi?$AAn?$AAg?$AA?5?$AAf?$AAF?$AAo?$AAr?$AAc?$AAe?$AA?5?$AAi?$AAn?$AA?5@ 10001d70     battdrvr_lib:battdrvr.obj
 0001:00000e00       ??_C@_1JA@JJAJNBB@?$AA?$CF?$AAs?$AA?3?$AA?5?$AAI?$AAO?$AAC?$AAT?$AAL?$AA?3?$AA0?$AAx?$AA?$CF?$AAx?$AA?0?$AA?5?$AAI?$AAn?$AAB?$AAu?$AAf?$AA?3?$AA0?$AAx?$AA?$CF?$AAx?$AA?0?$AA?5?$AAI?$AAn?$AAB?$AAu@ 10001e00     battdrvr_lib:battdrvr.obj
 0001:00000e90       ??_C@_1BE@PEIFHNGC@?$AAI?$AAO?$AAC?$AAo?$AAn?$AAt?$AAr?$AAo?$AAl?$AA?$AA@ 10001e90     battdrvr_lib:battdrvr.obj
 0001:00000ea4       ??_C@_1CO@KOJHAELC@?$AAO?$AAp?$AAe?$AAn?$AA?$CI?$AA?$CF?$AAx?$AA?0?$AA?5?$AA0?$AAx?$AA?$CF?$AAx?$AA?0?$AA?5?$AA0?$AAx?$AA?$CF?$AAx?$AA?$CJ?$AA?$AN?$AA?6?$AA?$AA@ 10001ea4     battdrvr_lib:battdrvr.obj
 0001:00000ed4       ??_C@_1BI@BIIJHOGM@?$AAC?$AAl?$AAo?$AAs?$AAe?$AA?$CI?$AA?$CF?$AAx?$AA?$CJ?$AA?$AN?$AA?6?$AA?$AA@ 10001ed4     battdrvr_lib:battdrvr.obj
 0001:00000eec       ??_C@_1O@OBHHKAKF@?$AAR?$AAe?$AAa?$AAd?$AA?$AN?$AA?6?$AA?$AA@ 10001eec     battdrvr_lib:battdrvr.obj
 0001:00000f00       ??_C@_1HO@LMJLIJKE@?$AA?$CK?$AA?$CK?$AA?$CK?$AA?5?$AAD?$AAL?$AAL?$AA_?$AAP?$AAR?$AAO?$AAC?$AAE?$AAS?$AAS?$AA_?$AAD?$AAE?$AAT?$AAA?$AAC?$AAH?$AA?5?$AA?9?$AA?5?$AAC?$AAu?$AAr?$AAr?$AAe?$AAn?$AAt@ 10001f00     battdrvr_lib:battdrvr.obj
 0001:00000f80       ??_C@_1HO@FJPAGEDH@?$AA?$CK?$AA?$CK?$AA?$CK?$AA?5?$AAD?$AAL?$AAL?$AA_?$AAP?$AAR?$AAO?$AAC?$AAE?$AAS?$AAS?$AA_?$AAA?$AAT?$AAT?$AAA?$AAC?$AAH?$AA?5?$AA?9?$AA?5?$AAC?$AAu?$AAr?$AAr?$AAe?$AAn?$AAt@ 10001f80     battdrvr_lib:battdrvr.obj
 0001:00001000       ??_C@_1BA@LEPJIIOK@?$AAU?$AAn?$AAk?$AAn?$AAo?$AAw?$AAn?$AA?$AA@ 10002000     battdrvr_lib:battapi.obj
 0001:00001010       ??_C@_1HI@BEOKGNLO@?$AAC?$AA?3?$AA?2?$AAy?$AAm?$AAz?$AAk?$AAi?$AA?2?$AAp?$AAu?$AAb?$AAl?$AAi?$AAc?$AA?2?$AAC?$AAO?$AAM?$AAM?$AAO?$AAN?$AA?2?$AAo?$AAa?$AAk?$AA?2?$AAd?$AAr?$AAi?$AAv?$AAe@ 10002010     battdrvr_lib:battapi.obj
 0001:000010b0       BatteryPDDInitialize       100020b0 f   battdrvr.obj
 0001:000010d8       BatteryPDDDeinitialize     100020d8 f   battdrvr.obj
 0001:00001150       BatteryPDDResume           10002150 f   battdrvr.obj
 0001:000011c8       BatteryPDDPowerHandler     100021c8 f   battdrvr.obj
 0001:00001248       BatteryPDDGetStatus        10002248 f   battdrvr.obj
 0001:00001300       BatteryPDDGetLevels        10002300 f   battdrvr.obj
 0001:0000138c       BatteryPDDSupportsChangeNotification 1000238c f   battdrvr.obj
 0001:00001418       BatteryThreadProc          10002418 f   battdrvr_lib:battdrvr.obj
 0001:000017d0       Init                       100027d0 f   battdrvr_lib:battdrvr.obj
 0001:00001f00       Deinit                     10002f00 f   battdrvr_lib:battdrvr.obj
 0001:00002110       IOControl                  10003110 f   battdrvr_lib:battdrvr.obj
 0001:00002cb0       PowerDown                  10003cb0 f   battdrvr_lib:battdrvr.obj
 0001:00002ccc       PowerUp                    10003ccc f   battdrvr_lib:battdrvr.obj
 0001:00002d08       Open                       10003d08 f   battdrvr_lib:battdrvr.obj
 0001:00002d70       Close                      10003d70 f   battdrvr_lib:battdrvr.obj
 0001:00002dd0       Read                       10003dd0 f   battdrvr_lib:battdrvr.obj
 0001:00002e44       Write                      10003e44 f   battdrvr_lib:battdrvr.obj
 0001:00002eb8       Seek                       10003eb8 f   battdrvr_lib:battdrvr.obj
 0001:00002ee0       DllMain                    10003ee0 f   battdrvr_lib:battdrvr.obj
 0001:00002fe0       GetCurrentThread           10003fe0 f i battdrvr_lib:battdrvr.obj
 0001:00002ff8       GetCurrentThreadId         10003ff8 f i battdrvr_lib:battdrvr.obj
 0001:00003024       SetEvent                   10004024 f i battdrvr_lib:battdrvr.obj
 0001:0000305c       GetCurrentProcess          1000405c f i battdrvr_lib:battdrvr.obj
 0001:00003074       GetCurrentProcessId        10004074 f i battdrvr_lib:battdrvr.obj
 0001:000030a0       BatteryAPIStopwatch        100040a0 f   battdrvr_lib:battapi.obj
 0001:00003200       BatteryAPIGetSystemPowerStatusEx2 10004200 f   battdrvr_lib:battapi.obj
 0001:000034c8       BatteryAPIGetSystemPowerStatusEx 100044c8 f   battdrvr_lib:battapi.obj
 0001:00003548       BatteryAPIGetLifeTimeInfo  10004548 f   battdrvr_lib:battapi.obj
 0001:00003624       add64_64_64                10004624 f   battdrvr_lib:battapi.obj
 0001:000036b4       sub64_64_64                100046b4 f   battdrvr_lib:battapi.obj
 0001:0000374c       BatteryAPINotifyOfTimeChange 1000474c f   battdrvr_lib:battapi.obj
 0001:000037c4       NKDbgPrintfW               100047c4 f   coredll:COREDLL.dll
 0001:000037d4       GetLastError               100047d4 f   coredll:COREDLL.dll
 0001:000037e4       WaitForSingleObject        100047e4 f   coredll:COREDLL.dll
 0001:000037f4       PowerPolicyNotify          100047f4 f   coredll:COREDLL.dll
 0001:00003804       CeSetThreadPriority        10004804 f   coredll:COREDLL.dll
 0001:00003814       __GetUserKData             10004814 f   coredll:COREDLL.dll
 0001:00003824       DeleteCriticalSection      10004824 f   coredll:COREDLL.dll
 0001:00003834       LocalFree                  10004834 f   coredll:COREDLL.dll
 0001:00003844       CloseHandle                10004844 f   coredll:COREDLL.dll
 0001:00003854       CreateThread               10004854 f   coredll:COREDLL.dll
 0001:00003864       LocalAlloc                 10004864 f   coredll:COREDLL.dll
 0001:00003874       RegCloseKey                10004874 f   coredll:COREDLL.dll
 0001:00003884       RegQueryValueExW           10004884 f   coredll:COREDLL.dll
 0001:00003894       OpenDeviceKey              10004894 f   coredll:COREDLL.dll
 0001:000038a4       CreateEventW               100048a4 f   coredll:COREDLL.dll
 0001:000038b4       InitializeCriticalSection  100048b4 f   coredll:COREDLL.dll
 0001:000038c4       OpenEventW                 100048c4 f   coredll:COREDLL.dll
 0001:000038d4       EventModify                100048d4 f   coredll:COREDLL.dll
 0001:000038e4       LeaveCriticalSection       100048e4 f   coredll:COREDLL.dll
 0001:000038f4       EnterCriticalSection       100048f4 f   coredll:COREDLL.dll
 0001:00003904       SetLastError               10004904 f   coredll:COREDLL.dll
 0001:00003914       CeSetPowerOnEvent          10004914 f   coredll:COREDLL.dll
 0001:00003924       DisableThreadLibraryCalls  10004924 f   coredll:COREDLL.dll
 0001:00003934       RegisterDbgZones           10004934 f   coredll:COREDLL.dll
 0001:00003944       GetTickCount               10004944 f   coredll:COREDLL.dll
 0001:00003954       SystemTimeToFileTime       10004954 f   coredll:COREDLL.dll
 0001:00003964       GetLocalTime               10004964 f   coredll:COREDLL.dll
 0001:00003974       FileTimeToSystemTime       10004974 f   coredll:COREDLL.dll
 0001:00003984       _DllMainCRTStartup         10004984 f   corelib0:pegdmain.obj
 0001:00003b2c       __security_init_cookie     10004b2c f   corelib0:seccinit.obj
 0001:00003bf4       exit                       10004bf4 f   corelib0:cexit.obj
 0001:00003d74       _exit                      10004d74 f   corelib0:cexit.obj
 0001:00003d98       _cexit                     10004d98 f   corelib0:cexit.obj
 0001:00003db4       _c_exit                    10004db4 f   corelib0:cexit.obj
 0001:00003dd0       _initterm                  10004dd0 f   corelib0:crt0dat.obj
 0001:00003e24       _cinit                     10004e24 f   corelib0:crt0dat.obj
 0001:00003e60       _onexit                    10004e60 f   corelib0:onexit.obj
 0001:00004164       atexit                     10005164 f   corelib0:onexit.obj
 0001:000041b8       memcmp                     100051b8 f   corelib1:COREDLL.dll
 0001:000041c8       memcpy                     100051c8 f   corelib1:COREDLL.dll
 0001:000041d8       memset                     100051d8 f   corelib1:COREDLL.dll
 0001:000041e8       __C_specific_handler       100051e8 f   corelib1:COREDLL.dll
 0001:000041f8       _XcptFilter                100051f8 f   corelib1:COREDLL.dll
 0001:00004208       __security_gen_cookie2     10005208 f   corelib1:COREDLL.dll
 0001:00004218       free                       10005218 f   corelib1:COREDLL.dll
 0001:00004228       malloc                     10005228 f   corelib1:COREDLL.dll
 0001:00004238       realloc                    10005238 f   corelib1:COREDLL.dll
 0001:00004248       _msize                     10005248 f   corelib1:COREDLL.dll
 0001:00004258       InterlockedExchange        10005258 f   coredll:COREDLL.dll
 0001:00004268       TerminateProcess           10005268 f   coredll:COREDLL.dll
 0001:00004278       InterlockedCompareExchange 10005278 f   coredll:COREDLL.dll
 0001:000043a0       __IMPORT_DESCRIPTOR_COREDLL 100053a0     coredll:COREDLL.dll
 0001:000043b4       __NULL_IMPORT_DESCRIPTOR   100053b4     coredll:COREDLL.dll
 0002:00000000       __imp_NKDbgPrintfW         10006000     coredll:COREDLL.dll
 0002:00000004       __imp_GetLastError         10006004     coredll:COREDLL.dll
 0002:00000008       __imp_WaitForSingleObject  10006008     coredll:COREDLL.dll
 0002:0000000c       __imp_PowerPolicyNotify    1000600c     coredll:COREDLL.dll
 0002:00000010       __imp_CeSetThreadPriority  10006010     coredll:COREDLL.dll
 0002:00000014       __imp___GetUserKData       10006014     coredll:COREDLL.dll
 0002:00000018       __imp_DeleteCriticalSection 10006018     coredll:COREDLL.dll
 0002:0000001c       __imp_LocalFree            1000601c     coredll:COREDLL.dll
 0002:00000020       __imp_CloseHandle          10006020     coredll:COREDLL.dll
 0002:00000024       __imp_CreateThread         10006024     coredll:COREDLL.dll
 0002:00000028       __imp_LocalAlloc           10006028     coredll:COREDLL.dll
 0002:0000002c       __imp_RegCloseKey          1000602c     coredll:COREDLL.dll
 0002:00000030       __imp_RegQueryValueExW     10006030     coredll:COREDLL.dll
 0002:00000034       __imp_OpenDeviceKey        10006034     coredll:COREDLL.dll
 0002:00000038       __imp_CreateEventW         10006038     coredll:COREDLL.dll
 0002:0000003c       __imp_InitializeCriticalSection 1000603c     coredll:COREDLL.dll
 0002:00000040       __imp_OpenEventW           10006040     coredll:COREDLL.dll
 0002:00000044       __imp_EventModify          10006044     coredll:COREDLL.dll
 0002:00000048       __imp_LeaveCriticalSection 10006048     coredll:COREDLL.dll
 0002:0000004c       __imp_EnterCriticalSection 1000604c     coredll:COREDLL.dll
 0002:00000050       __imp_SetLastError         10006050     coredll:COREDLL.dll
 0002:00000054       __imp_CeSetPowerOnEvent    10006054     coredll:COREDLL.dll
 0002:00000058       __imp_DisableThreadLibraryCalls 10006058     coredll:COREDLL.dll
 0002:0000005c       __imp_RegisterDbgZones     1000605c     coredll:COREDLL.dll
 0002:00000060       __imp_GetTickCount         10006060     coredll:COREDLL.dll
 0002:00000064       __imp_SystemTimeToFileTime 10006064     coredll:COREDLL.dll
 0002:00000068       __imp_GetLocalTime         10006068     coredll:COREDLL.dll
 0002:0000006c       __imp_FileTimeToSystemTime 1000606c     coredll:COREDLL.dll
 0002:00000070       __imp_memcmp               10006070     corelib1:COREDLL.dll
 0002:00000074       __imp_memcpy               10006074     corelib1:COREDLL.dll
 0002:00000078       __imp_memset               10006078     corelib1:COREDLL.dll
 0002:0000007c       __imp___C_specific_handler 1000607c     corelib1:COREDLL.dll
 0002:00000080       __imp__XcptFilter          10006080     corelib1:COREDLL.dll
 0002:00000084       __imp___security_gen_cookie2 10006084     corelib1:COREDLL.dll
 0002:00000088       __imp_free                 10006088     corelib1:COREDLL.dll
 0002:0000008c       __imp_malloc               1000608c     corelib1:COREDLL.dll
 0002:00000090       __imp_realloc              10006090     corelib1:COREDLL.dll
 0002:00000094       __imp__msize               10006094     corelib1:COREDLL.dll
 0002:00000098       __imp_InterlockedExchange  10006098     coredll:COREDLL.dll
 0002:0000009c       __imp_TerminateProcess     1000609c     coredll:COREDLL.dll
 0002:000000a0       __imp_InterlockedCompareExchange 100060a0     coredll:COREDLL.dll
 0002:000000a4       \177COREDLL_NULL_THUNK_DATA 100060a4     coredll:COREDLL.dll
 0002:000000a8       dpCurSettings              100060a8     battdrvr_lib:battzones.obj
 0002:000004ec       __security_cookie          100064ec     corelib0:seccinit.obj
 0002:000004f0       __security_cookie_complement 100064f0     corelib0:seccinit.obj
 0002:00000500       _exitflag                  10006500     corelib0:cexit.obj
 0002:00000504       v_imsStart                 10006504     <common>
 0002:00000508       v_fStopwatchRunning        10006508     <common>
 0002:00000510       v_ftLastChange             10006510     <common>
 0002:00000518       v_cmsPreviousCpuUsage      10006518     <common>
 0002:0000051c       v_fOnExternalPower         1000651c     <common>
 0002:00000520       v_cmsUsed                  10006520     <common>
 0002:00000540       gcsPddBuffer               10006540     <common>
 0002:00000560       gBatteryContext            10006560     <common>
 0002:000005a0       ghevResume                 100065a0     <common>
 0002:000005a4       gpfnBatteryPddIOControl    100065a4     <common>
 0002:000005c0       gcsBattery                 100065c0     <common>
 0002:000005d4       gpPddBufferTemp            100065d4     <common>
 0002:000005d8       gpPddBuffer                100065d8     <common>
 0002:000005dc       gdwPddBufferSize           100065dc     <common>
 0002:000005e0       gfExiting                  100065e0     <common>
 0002:000005e4       ghtBattery                 100065e4     <common>
 0002:000005e8       __onexitend                100065e8     <common>
 0002:000005ec       __onexitbegin              100065ec     <common>
 0002:000005f0       g_pcsExit                  100065f0     <common>
 0002:000005f4       _pRawDllMain               100065f4     <common>

 entry point at        0001:00003984

 Static symbols

 0001:000039d8       _DllMainCRTStartupHelper   100049d8 f   corelib0:pegdmain.obj
 0001:00003c18       doexit                     10004c18 f   corelib0:cexit.obj
 0001:00003ebc       lockexit                   10004ebc f   corelib0:onexit.obj
 0001:00003f58       unlockexit                 10004f58 f   corelib0:onexit.obj
 0001:00003f84       _onexit_nolock             10004f84 f   corelib0:onexit.obj
